:02000000632873
:0800080091000308920083122D
:100010000B11B13081001A201220442012088300F5
:10002000110809009F1C0800A1032108031D0800F6
:100030009F1008001F1C08009C031C08031D0800DB
:10004000C8309C0030209D031D08031D08003B3074
:100050009D009E0336201E08031D08001F10080087
:10006000A0193428A0150800A01108001E0895004A
:10007000DC200C3084000F308000840A16088000D9
:10008000840A1708800008008F0A0F08033A031932
:100090008F010C300F078400000890002008F83909
:1000A000A0000F085A200739A00420088500100876
:1000B000860008008207063405340334A1009F142B
:1000C0009F1860280800831285018601831681121B
:1000D0008111011081100115F03086008501831215
:1000E000FF3085008600A0008F01C8309C003C30A6
:1000F0009D008B01B13081008B168B171F10A0154E
:10010000FA203620BB201408023A0319902814085C
:10011000043A031997281408083A03199E288128DD
:100120009E0A1E083D3A031D81289E0381289E03D6
:100130001E08003A031D81289E0A81281F140121F0
:1001400032305E201F1CAA280608F039F03A031945
:10015000A2287E282012AE2020167E28201AB2283F
:100160002016B328201232305E200608F039F03A0B
:10017000031D0800AE280608F039F03A031DBB281D
:100180000608F039F03A0319C02804305E2006084A
:10019000F039F03A0319C52806089400940C940C21
:1001A000940C940C14090F3994000608F039F03AB5
:1001B000031DD5281408080015089A009B01083073
:1001C00099009A0D9B0D0A301B02031CEB280A3084
:1001D0009B020314031C0310960D990BE1280A30AF
:1001E0009900980116089807990BF228180815022B
:1001F000970008000030890083160814831208084D
:100200009E00003089001E0888000C218316881883
:10021000072908118312080083168B13081555301F
:0E0220008900AA30890088148B178312080009
:02400E0011009F
:024200000100BB
:00000001FF
